:100000000C94D3020C941A030C941A030C941A0344
:100010000C941A030C941A030C941A030C941A03EC
:100020000C941A030C941A030C94B71F0C94892097
:100030000C941A030C941A030C941A030C941A03CC
:100040000C941A030C94FC1A0C941A030C941A03C3
:100050000C941A030C9414160C941A030C941A039F
:100060000C941A030C941A030C941A030C941A039C
:100070000C941A030C941A030C941A030C941A038C
:100080000C941A030C941A030C941A030C941A037C
:100090000C941A030C941A030C941A030C941A036C
:1000A0000C941A030C941A030C941A03730C730C1B
:1000B000A20CA20CD80CF80C290E290E030D290E47
:1000C000B30DB30D1A0E290E290E230EC00DC00D4F
:1000D000C00DC00DC00DC00DC00DC00DC00DC00DB8
:1000E000C00DC00DC00DC00DC00DC00DD20DDF0D77
:1000F000E60DED0DF70DF620182106221821062237
:100100005D2180210622D521E821750A01E2012C1A
:10011000022C02E274FA011602160104020401091B
:1001200002090104020401150215010C020C012848
:10013000022800750A01E2012C022C02E274FA0185
:10014000170217010802080115021501100210011B
:100150000C020C0111021101040204010F020F0133
:1001600028022800750A01E2012C022C02E274FA2E
:100170000105020501050205010802080107020741
:10018000010C020C011702170128022800750A0150
:10019000E30116021602E301E3012B022B02E30145
:1001A000E30115021502E300750A01E301160216C8
:1001B00002E301E3012B022B02E3000000F0A12E79
:1001C000004C002A00E100E00000001E00140004C2
:1001D000001D00E200E2001F001A0016001B00E3F1
:1001E000002B00200008000700060050002C002112
:1001F000001500090019004F004B00220017000AEB
:1002000000050000003500015301510000E300002B
:10021000003400015301510000E3000000290023D5
:10022000001C000B00110000002A00240018000D23
:1002300000100052004E0025000C000E0036005148
:10024000002800260012000F0037002F002B002787
:10025000001300334238613000E0002D00310034DB
:1002600068E5002C00000001000100010001000110
:100270000000003A002F0036020100010001003B9F
:1002800000300037020100010001003C002F02266F
:10029000020100010001003D0030022702010001BF
:1002A0000001003E00340234002E00000001000175
:1002B0000001000000010000000100010001000039
:1002C000000100000001003F0038002D0033020053
:1002D0000001004000240021001E00270001004111
:1002E00000250022001F00370001004200260023E5
:1002F00000200050000100430025022E022E004F76
:10030000000100440045000100010001000000015F
:10031000000100010001000100000069000100016E
:10032000000100010001006A000100043001000129
:1003300000010001004B004E00010001000100011E
:100340000001300100010001004A000100033001FA
:100350000002300000010001000100000001000067
:100360000001001408010000000100000001001A53
:100370000830082F082C0200000100350A520C50EA
:10038000002C00A9004D00350852005100AC00AA15
:100390000019080100510C4F00AB00A8000608012D
:1003A0000001000100010001001B08A5000100AED2
:1003B000000100010000000000000000000000003B
:1003C0000000010204060A0F17202C3A4A5D7187CB
:1003D0009DB3C7DAE9F5FCFFFCF5E9DAC7B39D8701
:1003E000715D4A3A2C20170F0A0604020100000032
:1003F0000000000000000016034500720067006F57
:100400000044006F007800200045005A00000016EC
:10041000034500720067006F0044006F0078002001
:100420000045005A0000000403090409026D00049D
:100430000100A0FA090400000103010100092111D3
:100440000100012240000705810308000A09040198
:10045000000103010200092111010001224D0007E2
:1004600005820308000A09040200010300000009D4
:1004700021110100012236000705830308000A0943
:1004800004030001030000000921110100012239C9
:10049000000705840310000112011001000000088C
:1004A000EDFE071301000102000105010906A1018B
:1004B000050719E029E71500250195087501810256
:1004C0000508190129059505750191029501750326
:1004D0009101050719002977150025019578750107
:1004E0008102C005010980A101850216810026B79D
:1004F000001A81002AB700751095018100C0050C13
:100500000901A1018503160100269C021A01002A97
:100510009C02751095018100C005010902A1010925
:1005200001A1000509190129051500250195057589
:100530000181029501750381010501093009311519
:1005400081257F95027508810609381581257F95DB
:100550000175088106050C0A38021581257F950171
:1005600075088106C0C005010906A101050719E04B
:1005700029E7150025019508750181029501750887
:10058000810105081901290595057501910295015B
:10059000750391010507190029FF150026FF009535
:1005A0000675088100C011241FBECFEFDAE0DEBF60
:1005B000CDBF04B603FE27C08091010290910202D4
:1005C000A0910302B09104028730904BA740B04B3A
:1005D000D1F41092010210920202109203021092C2
:1005E000040214BE84B7877F84BF0FB6F894A89521
:1005F00080916000886180936000109260000FBE5F
:10060000E0E0FFE3099511E0A0E0B1E0E0EAF7E403
:1006100002C005900D92A433B107D9F712E0A4E30C
:10062000B1E001C01D92A130B107E1F70E94FC1CAE
:100630000C94CE230C9400001092B9008AE08093B1
:10064000B800089594EA9093BC009091BC0097FF85
:10065000FCCF9091B900987F983021F0903111F043
:1006600081E008958093BB0084E88093BC00809172
:10067000BC0087FFFCCF8091B900887F883111F0E2
:10068000803471F780E0089584E98093BC00809104
:10069000BC0084FDFCCF08958093BB0084E8809368
:1006A000BC008091BC0087FFFCCF9091B900987F7F
:1006B00081E0983209F480E0089584E88093BC00DA
:1006C0008091BC0087FFFCCF8091BB00089580B370
:1006D0008C7080BB81B3836F81BB089580910101D1
:1006E000811115C080E40E942203809301018111D1
:1006F0000CC082E10E944C0380930101811105C06E
:100700008FEF0E944C03809301010E94440384B147
:10071000807F84B985B1807F85B98AB1837F8AB9AA
:100720008BB1837F8BB93E98469808950C94E4046E
:100730000E942509809301010E946E030E946703B5
:10074000A5E3B1E0E3E4F1E08EE08E0F11921D929B
:100750008E13FCCF0C940F090E9425098093010190
:100760000E946E030E946703A5E3B1E0E3E4F1E0B9
:100770008EE08E0F11921D928E13FCCF0895BF92C2
:10078000CF92DF92EF92FF920F931F93CF93DF935D
:1007900080910101882379F0809134018F5F8093EB
:1007A0003401811108C00E94250980930101811143
:1007B00002C00E94B70805E311E0C0E0D0E0EE24DB
:1007C000E394F12CDD24D39495E0C92EC730D105F4
:1007D00000F58091010181113CC080E40E94220358
:1007E00080930101811112C082E10E944C03809329
:1007F000010181110BC0C7010C2E01C0880F0A94A2
:10080000EAF780950E944C03809301010E94440303
:1008100020C0CA30A1F028F4C83059F0C93061F0C6
:1008200005C0CC3089F070F0CD3089F0209A28983E
:1008300010C0219A29980DC0229A2A980AC0239A9A
:100840002B9807C0529A01C0539A5B9802C03E9AF7
:10085000469880EA8A95F1F7C730D10518F580915E
:100860000101811144C080E40E94220380930101B0
:10087000882311F0B12C12C083E10E944C038093B5
:1008800001018111F7CF81E40E94220380930101CD
:100890008111F0CF0E945D03B82EB0940E944403F2
:1008A0008B2D26C08FB181708D25799902C092E081
:1008B00001C090E0892B7C9902C024E001C020E0B7
:1008C000822B7D9902C028E001C020E0822B7E9916
:1008D00002C090E101C090E0892B9FB19095991FD3
:1008E0009927991F9295990F907E892B01C080E0DE
:1008F000F8019081981719F08083C09200010E943E
:100900006E0321960F5F1F4FCE30D10509F05ECFE9
:10091000809100018823A1F08150809300018823F9
:1009200029F0F5E0FA95F1F700000AC0A3E4B1E080
:10093000E5E3F1E0CF01825F91919D938E13FCCFAF
:100940000E94410681E0DF91CF911F910F91FF90AE
:10095000EF90DF90CF90BF900895E82FF0E0ED5B2F
:10096000FE4F808108950895FC016230B9F028F4AB
:10097000662341F0613061F023C06330A9F0643038
:10098000C9F01EC082818823D9F088EA91E00895D9
:1009900082818823A9F08DE891E0089582818823DF
:1009A00079F084E691E008958281882349F083E319
:1009B00091E008958281882319F08AE091E00895FA
:1009C00080E090E0089508956091B0017091B101C8
:1009D0008091B2019091B3010E94081556985E98DB
:1009E00025982D9826982E9827982F98813019F0C1
:1009F000823021F00895259A2D9A0895269A2E9AEC
:100A0000089581E0089581E008950C9403050E9403
:100A1000940E2FEF84E39CE0215080409040E1F75A
:100A200000C000000C9439160F931F93CF93DF93EF
:100A30008C01FC01C081D181CE010E948D13BE01C9
:100A40000E94D807EC01B8010E940505882309F42B
:100A500012C1B801CE010E946808882309F40BC1B5
:100A6000B801CE010E948109882309F404C1C43170
:100A7000F0E7DF0708F0CDC0C23080E7D80708F400
:100A8000A3C0F8018281882309F4AAC00E947215CC
:100A9000811102C00E9458150E94851590E0909324
:100AA000F3018093F201C230F0E7DF0721F4809177
:100AB000F201816082C0C33080E7D80721F48091C1
:100AC000F20182607AC0C430E0E7DE0721F4809151
:100AD000F201846072C0C530F0E7DF0719F480913D
:100AE000F20127C0C63080E7D80721F48091F201D7
:100AF000806163C0C730E0E7DE0721F48091F20136
:100B000080625BC0C830F0E7DF0721F48091F2011A
:100B1000806453C0C93080E7D80721F48091F20186
:100B200080684BC0CA30E0E7DE0729F48091F2010B
:100B30008460886042C0CB30F0E7DF0721F4809109
:100B4000F2018E7F3AC0CC3080E7D80721F4809143
:100B5000F2018D7F32C0CD30E0E7DE0721F48091D5
:100B6000F2018B7F2AC0CE30F0E7DF0719F48091C5
:100B7000F20122C0CF3080E7D80721F48091F20142
:100B80008F7E1BC0C031E0E7DE0721F48091F201C7
:100B90008F7D13C0C131F0E7DF0721F48091F201AE
:100BA0008F7B0BC0C231D04721F48091F2018F7747
:100BB00004C08091F2018B7F877F8093F201809146
:100BC000F2010E94891557C0C115E0E7DE0779F0F0
:100BD000C130D047A1F081E0809351018093520150
:100BE000C801DF91CF911F910F910C940105F8017D
:100BF0008281882309F43FC00E9407053CC0F801A8
:100C000082818823C1F18091CD0181608093CD01E3
:100C100032C0CB3380E7D807A1F4F8018281882362
:100C200021F01092510182E016C080915101811192
:100C300006C086E20E940C0B86E20E94DF0B82E077
:100C400018C0CC33D04739F6F8018281882331F0BF
:100C50001092520180E20E942E0C0DC08091520130
:100C6000811106C087E20E940C0B87E20E94DF0B15
:100C700080E20E94350C80E0DF91CF911F910F91AF
:100C800008950C94960308950C9443060C9444061E
:100C900026E0729FF001112444E5849FE00DF11DD0
:100CA0001124E60FF11DEE0FFF1FE154FE4F859159
:100CB00094910E94EA07811560E49607B0F58115CA
:100CC00070E3970708F0E6C0803E9105D8F4803CB9
:100CD000910508F06CC0883A910578F4853A910541
:100CE00008F06BC08130910509F460C108F417C1A8
:100CF0008430910508F05AC112C18D3B910508F46A
:100D000067C00DC18F3F910509F048F4803F910500
:100D100008F0B5C0883E910508F448C100C18115AE
:100D200020E2920708F0ADC00895811543E59407CD
:100D300090F4811562E5960708F0D0C0811571E541
:100D4000970708F0C6C0811520E5920708F0A5C0F6
:100D50009F70906A0895811545E59407D8F4811530
:100D600064E5960708F0D0C0482F4695469570E296
:100D7000479FA00111248370992721E030E0B90139
:100D800002C0660F771F8A95E2F7CB01842B952B63
:100D90009A680895811576E5970708F4BAC09C0112
:100DA00030562115304108F0BAC09F70B6C0FC0122
:100DB000EE0FFF1FE55CFF4F6AC0853A910509F40D
:100DC000B1C0863A910509F0B0C082E890E4089578
:100DD000883A910509F4ACC0893A910509F4ABC091
:100DE0008A3A910509F4AAC08B3A910509F4A9C081
:100DF0008C3A910509F4A8C08B3B910509F4A7C072
:100E00008C3B910509F4A6C08D3A910509F4A5C063
:100E1000803B910509F4A4C08E3A910509F4A3C062
:100E20008F3A910509F4A2C0813B910509F4A1C054
:100E3000823B910509F4A0C0833B910509F49FC052
:100E4000843B910509F49EC0853B910509F49DC042
:100E5000863B910509F49CC0873B910509F49BC032
:100E6000883B910509F49AC0893B910509F499C022
:100E70008A3B910509F498C080E094E40895906558
:100E80000895FC01FF70EE0FFF1FE554FE4F8591A2
:100E9000949108959927906C0895482F437021E00C
:100EA00030E002C0220F331F4A95E2F73C68AC01E4
:100EB00064E0569547956A95E1F74370342B8F703F
:100EC0008695869560E2869FC0011124822B932B24
:100ED0000895982F8827816F906A0895482F469526
:100EE000469570E2479FA00111248370992721E065
:100EF00030E0B90102C0660F771F8A95E2F7CB0197
:100F0000842B952B9C680895982F8827846F906A6E
:100F100008958F719927982F88279062089580E00F
:100F200090E0089581E890E4089583E890E40895BE
:100F300082EE94E4089589EE94E408958AEE94E4B0
:100F4000089585EB94E4089586EB94E4089583EB8B
:100F500094E4089584EB94E4089587EB94E4089571
:100F60008CEC94E408958DEC94E4089583E895E482
:100F700008958AE895E4089582E995E4089584E95E
:100F800095E4089581E296E4089583E296E4089555
:100F900084E296E4089585E296E4089586E296E474
:100FA000089587E296E408958AE296E40895089504
:100FB00096E0799FF001112494E5899FE00DF11DE1
:100FC0001124E60FF11DEE0FFF1FE154FE4F859136
:100FD000949108958238910549F1B0F481339105D7
:100FE00009F458C048F48932910509F44EC08A3298
:100FF000910509F454C008958533910509F440C062
:101000008933910599F00895833E910529F138F4CB
:10101000803E910591F0823E9105A1F00895863EB3
:101020009105F9F0873E910531F108952091F20183
:1010300020FD3AC021FD38C008958091F20180FD65
:1010400035C032C08091F20182FF32C08091F2013E
:1010500084FD30C083EE39C08091F20182FD28C04A
:10106000F5CF8091F20183FF27C08091F20184FDCA
:1010700021C087EE2AC08091F20183FD1DC0F5CF0B
:101080008091F20185FD1AC01BC08091F20185FD9F
:1010900017C014C08091F20186FD14C015C0809164
:1010A000F20186FD11C00EC080EE0FC089E30DC0B5
:1010B00082EE0BC080E009C086EE07C089E205C061
:1010C00085E303C08AE201C081E390E008950895BA
:1010D0000F931F93CF93FB012281211102C0C1E026
:1010E00041C08C01C0916001C11125C0843190477D
:1010F000B1F70E94670881E0809360010E94DE15CD
:1011000090935F0180935E011092530110925501FC
:1011100010925401109257011092560110925901E9
:101120001092580110925B0110925A0110925D01C9
:1011300010925C0117C080915E0190915F010E9446
:10114000EA15883C910558F690915301E92FF0E09B
:10115000EE0FFF1FEC5AFE4F118300839F5F9093A9
:101160005301C0E08C2FCF911F910F910895569895
:101170005E9825982D9826982E9827982F988FEF6F
:1011800090E0909389008093880090938B008093E7
:101190008A0090938D0080938C00259A2D9A2FEFD2
:1011A00080E792E0215080409040E1F700C00000CD
:1011B000269A2E9A2FEF80E792E0215080409040AF
:1011C000E1F700C00000279A2F9A2FEF80E792E006
:1011D000215080409040E1F700C0000025982D98F4
:1011E0002FEF80E792E0215080409040E1F700C06F
:1011F000000026982E982FEF80E792E02150804043
:101200009040E1F700C0000027982F9856985E980C
:1012100025982D9826982E9827982F98089589EA32
:101220008093800089E08093810024982C983F98D7
:101230008AB18F748AB96E98479A8BB1806B8BB9DB
:10124000769A0E94B7080C94E30480E2809301012F
:101250008091610181110EC00E941C0381E0809386
:1012600061012FEF83ED90E3215080409040E1F742
:1012700000C0000080E40E942203809301018111DC
:101280002EC00E944C0380930101811128C00E944E
:101290004C0380930101811122C08FE30E944C0313
:1012A0008093010181111BC00E94440380E40E94CD
:1012B000220380930101811112C08CE00E944C0333
:1012C0008093010181110BC00E944C0380930101A6
:1012D000811105C08FE30E944C03809301010E949D
:1012E0004403809101010895282F882339F090E06C
:1012F0002A3010F44D9608950697089587E290E0FD
:101300000895FF920F931F93CF93DF93813020E8CE
:10131000920708F44DC0FB012281222309F448C042
:10132000EC01DF7780916201813079F050F08230FA
:10133000C1F482EE0E940C0B87E50E940C0B87E53E
:101340000EC082EE0E940C0B0CC080EE0E940C0BB3
:1013500081EE0E940C0B88E10E940C0B88E10E9438
:10136000DF0B0CE010E0CE01002E02C096958795B1
:101370000A94E2F78F700E947409F82E0E940C0BF9
:101380008F2D0E94DF0B045011090C3FFFEF1F0748
:1013900051F780916201813029F010F0823041F4E0
:1013A00082EE04C080EE0E94DF0B81EE0E94DF0B14
:1013B00081E0DF91CF911F910F91FF90089590935D
:1013C0006801809367010895E0916701F0916801D9
:1013D000309721F00190F081E02D099480E008958C
:1013E000E0916701F0916801309721F00280F3816C
:1013F000E02D09940895E0916701F091680130971C
:1014000021F00480F581E02D099408952091650173
:10141000309166018217930771F090936601809373
:101420006501E0916701F0916801309721F0068035
:10143000F781E02D099408952091630130916401B2
:101440008217930771F09093640180936301E09198
:101450006701F0916801309721F00084F185E02D5B
:101460000994089508950C94320A0E94D5150E949B
:1014700098030C945B16CF92DF92EF92FF920F933A
:101480001F93CF93DF93CDB7DEB72B970FB6F894AA
:10149000DEBF0FBECDBF0E94BF038AE6C82E81E02B
:1014A000D82E00E010E0E02E802F0E94AD04F6015F
:1014B00041916F01F42EF826B1F40F5F1F4F0E30EB
:1014C000110589F78FEF89838A831B820E94DE15BD
:1014D0008160782F9D838C8349815A816B818D81B6
:1014E0000E94DE0A40C09091CD0191FF04C08B871D
:1014F0000E94B3048B8520E030E04F2D50E0922F06
:10150000BA01022E02C0759567950A94E2F760FF52
:1015100024C02E83EF8221E030E0690102C0CC0CB0
:10152000DD1C9A95E2F790E08C219D21892B09F42E
:1015300020E028870E94DE158160782F9A878987AE
:101540004E815F8168858A850E94DE0AF801E6592E
:10155000FE4F8081C826C08206C02F5F3F4F2630D5
:10156000310569F6AACF0E94F317109169010E9414
:10157000E4091817A1F00E94E409809369012B96F1
:101580000FB6F894DEBF0FBECDBFDF91CF911F9194
:101590000F91FF90EF90DF90CF900C9446062B9622
:1015A0000FB6F894DEBF0FBECDBFDF91CF911F9174
:1015B0000F91FF90EF90DF90CF900895CF93DF933E
:1015C000CDB7DEB72B970FB6F894DEBF0FBECDBFF9
:1015D0004F83588769877A878B87DE01119686E06B
:1015E000FD0111928A95E9F785E0FE013796019099
:1015F0000D928A95E1F749815A816B817C818D81B9
:101600009E810E9432112B960FB6F894DEBF0FBE5A
:10161000CDBFDF91CF910895CF93882309F4CDC03A
:10162000C82F823859F40E94E40981FDC6C089E3BD
:101630000E940C140E94D91489E30CC0833879F4F9
:101640000E94E40980FDB9C083E50E940C140E9449
:10165000D91483E50E944E14CF910C94D914843888
:1016600059F40E94E40982FDA8C087E40E940C148A
:101670000E94D91487E4EECF8CEF8C0F813A48F4A6
:101680008C2F0E943D1A811198C08C2F0E940C143F
:10169000E3CF80E28C0F883048F4C77081E001C04E
:1016A000880FCA95EAF70E949214D6CF8BE58C0F6B
:1016B000833078F4C53A29F0C63A31F083E890E0F7
:1016C00005C081E890E002C082E890E0CF910C94E0
:1016D000060A88E58C0F853108F06FC0C83A61F1C1
:1016E000C93A69F1CA3A71F1CB3A79F1CC3A81F150
:1016F000CB3B89F1CC3B91F1CD3A99F1C03BA1F1C3
:10170000CE3AA9F1CF3AB1F1C13BB9F1C23BC1F137
:10171000C33BC9F1C43BD1F1C53BD9F1C63BE1F1B3
:10172000C73BE9F1C83BF1F1C93BF9F1CA3B09F408
:101730003FC080E090E03EC082EE90E03BC089EE8A
:1017400090E038C08AEE90E035C085EB90E032C082
:1017500086EB90E02FC083EB90E02CC084EB90E010
:1017600029C087EB90E026C08CEC90E023C08DEC84
:1017700090E020C083E891E01DC08AE891E01AC0A3
:1017800082E991E017C084E991E014C081E292E01F
:1017900011C083E292E00EC084E292E00BC085E2C9
:1017A00092E008C086E292E005C087E292E002C0C3
:1017B0008AE292E0CF910C941C0ACF91089588237D
:1017C00009F44BC0823859F40E94E40981FF45C0F6
:1017D00089E30E940C140E94D91489E30CC0833859
:1017E00071F40E94E40980FF38C083E50E940C1464
:1017F0000E94D91483E50E944E140C94D9148438A5
:1018000059F40E94E40982FF28C087E40E940C1466
:101810000E94D91487E4EFCF9CEF980F913A58F3C8
:1018200090E2980F983050F4877091E001C0990FC2
:101830008A95EAF7892F0E949814DFCF9BE5980FCD
:10184000933020F480E090E00C94060A885A8531A9
:1018500020F480E090E00C941C0A0895882321F085
:101860000E9492140C94D9140895882321F00E94A8
:1018700098140C94D91408957F928F929F92AF92EE
:10188000BF92CF92DF92EF92FF920F931F93CF936D
:10189000DF931F92CDB7DEB77C01C62E772EFC01F9
:1018A000058102950F70128111110E94AF140E94E0
:1018B0000514882379F0112369F080E28C0D8830BB
:1018C00048F082E00E94EE130E94051491E0D82EA9
:1018D000D92601C0D12CE72DE295EF70F0E0EA5A4D
:1018E000FF4F0C947F23872D807F072D0F70882357
:1018F00011F00295007F112389F0002309F490C1B3
:1019000080E28C0D883020F4802F0E94921403C056
:10191000802F0E94A2140E94D91482C18C2D0E9493
:10192000DF0B002309F495C180E28C0D883020F490
:10193000802F0E94981403C0802F0E94A8140E9438
:10194000D91487C1972D907F872D8F70903211F019
:101950008295807FCC2021F0F1E0CF16B1F01EC03F
:10196000112349F0002309F414C1013009F011C119
:101970000E94C2146EC1002319F0013009F469C13C
:1019800089830E94C51489810AC1112321F0023084
:1019900008F05FC1FEC001115CC101C1112321F03B
:1019A000002309F4F6C03CC1002309F4F8C03EC18D
:1019B000872D86958695837090E0009719F00197A2
:1019C00061F047C1112321F08C2D972D937002C037
:1019D00080E090E00E94060A3CC1112321F08C2D8A
:1019E000972D937002C080E090E00E941C0A31C1E4
:1019F0008C2D112319F00E94FB1602C00E94631760
:101A00000E94E81726C1872D837009F052C011117A
:101A100020C18C2D829586958770880F880F9C2D0C
:101A20009F70892E912CA12CB12C082E04C0880CFB
:101A3000991CAA1CBB1C0A94D2F7C4FE14C00FE068
:101A400010E020E030E0B901A80104C0440F551FA8
:101A5000661F771F8A95D2F7CB01BA016095709502
:101A60008095909503C060E070E0CB01272D26950E
:101A70002695237030E02230310569F0233031059E
:101A800089F0682979298A299B292130310571F04B
:101A90000E947A12DEC0682979298A299B290E942E
:101AA0009612D7C00E947A12C501B4010E945E123C
:101AB000D0C0112319F0872D817001C0869588232D
:101AC00009F4C7C08C2D829586958770880F880F82
:101AD0009C2D9F70892E912CA12CB12C082E04C016
:101AE000880C991CAA1CBB1C0A94D2F7C4FE14C013
:101AF0000FE010E020E030E0B901A80104C0440F7D
:101B0000551F661F771F8A95D2F7CB01BA016095E2
:101B100070958095909503C060E070E0CB01272D13
:101B2000269526952370422F50E04230510569F0EA
:101B30004330510589F0682979298A299B29413048
:101B4000510571F00E94541384C0682979298A29AB
:101B50009B290E9470137DC00E945413C501B401DB
:101B60000E94381376C08C2D90E0FC01E05EF109F4
:101B7000E531F10508F050C0EA59FF4F0C947F237E
:101B80000C2D0F70872D8F71112331F00E94D1120F
:101B9000802F0E942E0C5DC00E94F212802F0E94A6
:101BA000350C57C0112339F0011153C0872D8F71A7
:101BB0000E9417134EC0023008F04BC0F7CF11231C
:101BC00039F0872D8F710E94D11243C01123C9F3C0
:101BD000872D8F710E94F2123CC0112329F0872DAE
:101BE0008F710E94BC1235C00E94B21232C0112304
:101BF00051F0172D1F71812F0E94D11263E0812FA8
:101C00000E94E51326C081E00E94EE13023008F125
:101C100082E00E94EE131DC0112331F0002389F2EF
:101C20008C2D0E940C0B15C0002391F28C2D0E946C
:101C3000DF0B0FC0472D4F706C2DC7010E94B404FD
:101C40000E94D61106C0472D4F706C2DC7010E940F
:101C5000D707DD20F9F00E94E11380FD1BC0F701DA
:101C600012820E94DB130E94D112C7010E94590EFA
:101C70000E94DB130F90DF91CF911F910F91FF9086
:101C8000EF90DF90CF90BF90AF909F908F907F901C
:101C90000C94F2120F90DF91CF911F910F91FF9052
:101CA000EF90DF90CF90BF90AF909F908F907F90FC
:101CB00008950F931F93CF93DF93EC01888199814F
:101CC0002B813C81232BB9F09F3F11F48F3F99F07A
:101CD000CE010E941405882371F0688179818A8180
:101CE0000E94D7138C010E948C130E945312B801DA
:101CF000CE010E943C0CDF91CF911F910F9108956E
:101D00000E94AF140E94BF140E9484140E94D91430
:101D10000E9499180E94E81780E090E00E94060A4D
:101D200080E090E00C941C0A0E949F140C94800E9A
:101D30000E94CC13292F22952F7030E02C303105D2
:101D40004CF42A3031056CF422503109223031052F
:101D5000A8F407C02C30310569F02F30310551F05F
:101D60000DC0803F69F018F4803E40F409C0843F04
:101D700029F406C093FB882780F9089580E0089530
:101D800081E00895CF93DF9300D000D01F92CDB7AC
:101D9000DEB70F900F900F900F900F90DF91CF91C3
:101DA0000895CF93DF9300D000D000D0CDB7DEB739
:101DB00026960FB6F894DEBF0FBECDBFDF91CF9150
:101DC00008951F93CF93DF93C091780116E080911F
:101DD0007901C81799F0D0E01C9FF0011D9FF00D0C
:101DE0001124E658FE4F40815181628173818481C4
:101DF00095810E94D10E2196C770E9CFDF91CF91D6
:101E00001F9108954091AA015091AB016091AC01DE
:101E10007091AD018091AE019091AF010C94D10E03
:101E20008091AF0182958F7009F054C08091AC0110
:101E3000882309F44FC080917801A09179016091C5
:101E4000AA017091AB014091AD015091AE01B6E095
:101E50008A1709F43FC090E041155105C1F17F3F59
:101E600011F46F3FA1F1B89FF001B99FF00D11245B
:101E7000E658FE4F218172132AC02081621327C0C9
:101E80002281211124C0238134812417350710F4C5
:101E900021503109241B350B283C3105C0F4209119
:101EA000AF012F7020612093AF0126E0289FF00141
:101EB000299FF00D1124E158FE4F80818F708061C1
:101EC00080838AEA91E00E94590E0C94E10E0196FB
:101ED0008770BECF0895CF92DF92EF92FF920F935B
:101EE0001F93CF93DF93CDB7DEB762970FB6F89409
:101EF000DEBF0FBECDBF8C0185E0F801DE011D966F
:101F000001900D928A95E1F7D8014C9111965C9160
:101F1000119712966C9112971396CD90DC901497AE
:101F20003091AA017091AB018091AD019091AE0109
:101F3000009709F46BC17F3F19F43F3F09F466C174
:101F4000E090AC01EE2009F4C0C02091AF01C816AA
:101F5000D90628F0F601E81BF90BCF0104C08095E3
:101F600090958C0D9D1DFF24F394883C910578F08D
:101F7000F12C207F09F0C6C07C2DD98AC88A8989B6
:101F80000E94C20E8AEA91E00E94590EB1C0822FCF
:101F9000807F09F046C0751314C0341312C061115C
:101FA00010C02F7020612093AF010E94020F8AEAB7
:101FB00091E00E94590E8091AF01D80115968C9343
:101FC0002EC0CD2819F15F3F11F44F3FF9F0F62EE6
:101FD00061111CC0809178012091790136E082174F
:101FE00009F45AC090E0389FF001399FF00D112498
:101FF000E658FE4F7181571306C07081471303C026
:102000007281711103C001968770E9CFF62E6623A5
:1020100009F418C18091AF0181608093AF01F12C68
:1020200011C1751308C0341306C0611104C080913A
:10203000AF01D801C3C04D875E878D859E856A8BB1
:102040000E94980E6A898823E1F16623D1F12091DC
:10205000AF01822F82958F7090E0029774F080918B
:10206000AA019091AB0198878F831986DB86CA8677
:102070002C87CE0107960E94590E86E0F801AAEA45
:10208000B1E001900D928A95E1F70E94100F0E9435
:10209000020FFF24F394D6C04D875E878D859E8501
:1020A0000E94CC13292F22952F7030E02230310569
:1020B0000CF0BCC09F7009F0B6C0805E883008F498
:1020C000C1C0C8010E94590EE4CFC816D90608F451
:1020D00053C0F601E81BF90BCF01883C910508F4C9
:1020E00050C0F12C7C2DD98AC88A89890E94C20EE1
:1020F000EAEAF1E086E0DF011D928A95E9F70E94A5
:10210000020FA0C0751314C0341312C0611110C0A7
:102110008091AF01F8018583C8010E94590E86E0C5
:10212000EAEAF1E0DF011D928A95E9F7FE2C8AC008
:102130004D875E878D859E856A8B0E94980E6A8981
:10214000882309F4BECF662309F4BBCF2091AF01E9
:10215000822F82958F7090E002970CF48ECF809141
:10216000AA019091AB019A8389831B82DD82CC8284
:102170002E83CE0101967FCF809590958C0D9D1D6D
:10218000ACCFF62E662309F49CCF75132EC0341302
:102190002CC02091AF0120FD1FC0822F82958F702F
:1021A000D9F0D80115962C9315978F3049F08F5F91
:1021B000982F9295907F822F8F70892B15968C93F4
:1021C000C8010E94590E86E0F801AAEAB1E0019028
:1021D0000D928A95E1F793CF86E0F801AAEAB1E083
:1021E00001900D928A95E1F72DC04D875E878D8510
:1021F0009E850E94980E811140CF8091AF01816031
:102200008093AF01C8010E94590E1CC0662309F4D7
:1022100058CF4D875E878D859E850E94980E8823B6
:1022200009F44FCF2ACF811148CF0CC0243031059B
:102230000CF047CF9F7009F440CFF8019581907F53
:1022400009F03BCF8F2D62960FB6F894DEBF0FBE1C
:10225000CDBFDF91CF911F910F91FF90EF90DF9055
:10226000CF9008951F93CF93DF93CDB7DEB72C9710
:102270000FB6F894DEBF0FBECDBF4F835887698776
:102280007A878B879C87CE0107960E946B0F8823E5
:1022900069F08F8198852A853B85232BF1F19F3F3B
:1022A00009F063C08F3F09F060C037C086E0FE01CF
:1022B0003796DE01119601900D928A95E1F76F81B4
:1022C0007885EA85FB85309741F17F3F11F46F3FB8
:1022D00021F12091790130E0C90101968770992799
:1022E0004091780150E08417950709F447C069834D
:1022F0007A83FD83EC8396E0929FD001939FB00D8B
:102300001124A658BE4FFE01319601900D929A9568
:10231000E1F7809379010E94E10E16E08091780147
:10232000909179018917C1F1189FC0011124865835
:102330009E4F0E946B0F882379F1E09178011E9FD8
:10234000F0011124E658FE4F408151816281738172
:10235000848195810E94D10E8091780190E0019650
:102360008770992780937801D9CF4F8158856985E7
:102370007A858B859C850E94D10ECFCF0E94940ECA
:102380001092790110927801EAEAF1E086E0DF012B
:102390001D928A95E9F7C1CF2C960FB6F894DEBF4F
:1023A0000FBECDBFDF91CF911F910895EF92FF92A5
:1023B0000F931F93CF93DF938C01892B09F46CC08B
:1023C000F12CEE24E394E8012196F80184918437FE
:1023D00040F4843008F051C0813081F0823019F12E
:1023E0005BC0853709F444C0A8F19CE7980F90378B
:1023F00008F052C08F770E94DF0B41C00E5F1F4F65
:10240000FE01C49180E28C0F883048F4C7708E2D95
:1024100001C0880FCA95EAF70E94B21414C08C2F2D
:102420000E940C0B2DC00E5F1F4FFE01C49180E275
:102430008C0F883058F4C7708E2D01C0880FCA9554
:10244000EAF70E94B8140E94D9141AC08C2F0E9477
:10245000DF0B16C00E5F1F4FFE01C491CC2381F02D
:102460008FE99FE00197F1F700C00000C150F6CF5F
:102470000E5F1F4FFE01F49003C00E940C0B8E01F3
:102480008F2D882309F49FCFEFE9FFE03197F1F713
:1024900000C000008150F5CFDF91CF911F910F91C7
:1024A000FF90EF90089508956093B4017093B50183
:1024B0008093B6019093B7010C94800E0F931F93F5
:1024C0000091B4011091B5012091B6013091B7018E
:1024D000DC01CB01802B912BA22BB32B8093B40179
:1024E0009093B501A093B601B093B7011F910F91DE
:1024F0000C94800E0F931F930091B4011091B501BD
:102500002091B6013091B701DC01CB0180239123EA
:10251000A223B3238093B4019093B501A093B60195
:10252000B093B7011F910F910C94800E0F931F93DE
:102530000091B4011091B5012091B6013091B7011D
:10254000DC01CB0180279127A227B3278093B40118
:102550009093B501A093B601B093B7011F910F916D
:102560000C94800E1092B0011092B1011092B20141
:102570001092B3010C94800E41E050E060E070E0F6
:1025800004C0440F551F661F771F8A95D2F74093EA
:10259000B0015093B1016093B2017093B3010C94F8
:1025A000800E41E050E060E070E004C0440F551F31
:1025B000661F771F8A95D2F78091B0019091B10183
:1025C000A091B201B091B301482B592B6A2B7B2B00
:1025D0004093B0015093B1016093B2017093B30185
:1025E0000C94800E41E050E060E070E004C0440FC5
:1025F000551F661F771F8A95D2F7409550956095B5
:1026000070958091B0019091B101A091B201B0910B
:10261000B301482359236A237B234093B00150938D
:10262000B1016093B2017093B3010C94800E41E04C
:1026300050E060E070E004C0440F551F661F771F34
:102640008A95D2F78091B0019091B101A091B20129
:10265000B091B301482759276A277B274093B001DF
:102660005093B1016093B2017093B3010C94800E4A
:102670000F931F930091B0011091B1012091B2010D
:102680003091B301DC01CB01802B912BA22BB32B1A
:102690008093B0019093B101A093B201B093B301C4
:1026A0001F910F910C94800E0F931F930091B00116
:1026B0001091B1012091B2013091B301DC01CB0145
:1026C00080239123A223B3238093B0019093B1017F
:1026D000A093B201B093B3011F910F910C94800E9F
:1026E0000F931F930091B0011091B1012091B2019D
:1026F0003091B301DC01CB0180279127A227B327BA
:102700008093B0019093B101A093B201B093B30153
:102710001F910F910C94800E0895CF92DF92EF924B
:10272000FF920F931F93CF93DF938C01C090B4015E
:10273000D090B501E090B601F090B7018091B00162
:102740009091B101A091B201B091B301C82AD92AE8
:10275000EA2AFB2ACFE1D0E0D701C6010C2E04C043
:10276000B695A795979587950A94D2F780FF06C0EE
:10277000B8018C2F0E944806019721F4219760F739
:1027800080E001C08C2FDF91CF911F910F91FF90BE
:10279000EF90DF90CF900895CF93DF93EC010E94EC
:1027A0008D13BE010E944806DF91CF910895CB01A1
:1027B0000E94CC1308958091B801859585958595E3
:1027C00008958091B8018770089598E0899F9001DD
:1027D0001124262B2093B8010C94D1122091B8011A
:1027E000809582238093B801982F977069F430E028
:1027F000482F552747FD50952417350729F0859513
:10280000859585950C94F21208959091B801977072
:1028100081E009F480E0089590911501992321F059
:1028200090910201911109C020910301309104019E
:10283000F90132969FEF40E01FC0982F969596952C
:1028400096959F3050F5E0910301F0910401E90F56
:10285000F11D877021E030E0A90102C0440F551F2F
:102860008A95E2F7CA019181892B818308959F3F60
:1028700039F04F5F4E3041F051915813F8CF0DC0F1
:102880005111F7CF942FF5CF9F3F39F0F901E90FA0
:10289000F11D97FDFA958283089508959091150191
:1028A000992321F090910201911109C02091030117
:1028B00030910401F9013296205F3F4F1FC0982FDD
:1028C0009695969596959F30F0F4E0910301F091DE
:1028D0000401E90FF11D877021E030E0A90102C079
:1028E000440F551F8A95E2F7CA018095918189238B
:1028F000818308953196E217F30729F090819813A8
:10290000F9CF1082F7CF089581E090E0E0910301C4
:10291000F0910401E80FF91F1082019680319105B2
:10292000A9F708959091CC01892B8093CC0108954B
:1029300080959091CC0189238093CC0108951092C9
:10294000CC0108959091CB01892B8093CB01089500
:1029500080959091CB0189238093CB0108951092AB
:10296000CB0108959091CA01892B8093CA010895E3
:1029700080959091CA0189238093CA01089510928D
:10298000CA0108958093B90108951092B90108957C
:102990008091030190910401FC0131969C01205F1C
:1029A0003F4F80E0919191118F5FE217F307D1F7CC
:1029B0000895E0910301F09104018091CC0180839E
:1029C000E0910301F091040190818091CB01892B6A
:1029D0008083E0910301F091040190818091CA010C
:1029E000892B80838091B901882361F0E0910301F4
:1029F000F09104019081892B80830E94C814811179
:102A00001092B90180910301909104010C94F00996
:102A1000CF92DF92EF92FF926C01EE24FF24C1145B
:102A2000D104E104F10421F0C701B60120E101C0A5
:102A300020E0C72ED82EE92EFF24C114D104E104D2
:102A4000F10419F0285FC701B6016B017C0154E065
:102A5000F694E794D794C7945A95D1F7C114D1044A
:102A6000E104F10419F02C5FC701B6016B017C0190
:102A700042E0F694E794D794C7944A95D1F7C114ED
:102A8000D104E104F10419F02E5FC701B601DC01A5
:102A9000CB01B695A79597958795892B8A2B8B2B7C
:102AA00009F02F5F822FFF90EF90DF90CF90089575
:102AB0006DEE7EEF80E090E00E94B82360E082E05F
:102AC00090E00E94A72360E083E090E00E94A723AB
:102AD00060E084E090E00E94A72360E085E090E061
:102AE0000C94A72380E090E00E94A12321E08D3E7A
:102AF0009E4F09F020E0822F089582E090E00C9430
:102B0000992383E090E00C94992384E090E00C9466
:102B10009923682F84E090E00C94A7238091F8011A
:102B2000843039F11092CE0120E488E190E00FB6B4
:102B3000F894A895809360000FBE2093600080E019
:102B40000E94460683B7817F846083BF83B781601C
:102B500083BF7894889583B78E7F83BF0FB6F89430
:102B6000A895809160008861809360001092600059
:102B70000FBE08950895CF930E94AC030E94BF0337
:102B80000E94BA15C0E08C2F0E94AD04811104C0D0
:102B9000CF5FCE30C1F701C081E0CF9108950E9490
:102BA000940E0E94E4090C94460682E084BD93E0F2
:102BB00095BD9AEF97BD80936E0008952FB7F89456
:102BC0008091CF019091D001A091D101B091D2011B
:102BD0002FBF0895CF92DF92EF92FF920F931F9332
:102BE0002FB7F8944091CF015091D0016091D1015D
:102BF0007091D2012FBF6A017B01EE24FF248C016A
:102C000020E030E0C016D106E206F30610F4415091
:102C100051099A01281B390BC9011F910F91FF908F
:102C2000EF90DF90CF9008951F920F920FB60F9202
:102C300011248F939F93AF93BF938091CF01909175
:102C4000D001A091D101B091D2010196A11DB11D79
:102C50008093CF019093D001A093D101B093D20182
:102C6000BF91AF919F918F910F900FBE0F901F90CA
:102C700018950E943C1FF8942FEF87EA91E62150A7
:102C800080409040E1F700C0000087E090EBDC015D
:102C90008093010290930202A0930302B093040276
:102CA0009CE088E10FB6F894A895809360000FBE71
:102CB00090936000FFCF0E947215811102C00E94A4
:102CC00058150E947D158093CD010E94851590E0D6
:102CD0009093F3018093F20187FB882780F980931A
:102CE00002010E948115682F70E080E090E00C9452
:102CF00054128091D50180FF0BC06091080185E0DE
:102D0000689FB001112475956795759567952BC0DF
:102D100081FF09C06091080185E0689FB00111241E
:102D20007595679520C082FF07C06091080185E016
:102D3000689FB001112417C09091D6019923D1F05A
:102D400060910701961788F72091080185E0289F78
:102D500090011124929FA001939F500D112470E0C7
:102D6000CA010E946B236038710540F4611571053A
:102D700039F002C065E070E0862F08958FE708956E
:102D800081E008958091D50180FF08C0609106011F
:102D900070E0759567957595679521C081FF06C0B0
:102DA0006091060170E07595679519C082FF04C0B7
:102DB0006091060170E010C09091D6019923C1F096
:102DC000609105019617A0F780910601899FC001C7
:102DD000112470E00E946B236038710528F461159E
:102DE000710521F0862F08958FE7089581E00895F9
:102DF00061E070E0F4CF803F21F40E947916819564
:102E000004C0813F29F40E9479168093D901089566
:102E1000823F21F40E947916819504C0833F29F4F2
:102E20000E9479168093D8010895893F19F40E9471
:102E3000C21605C08A3F31F40E94C2168195809364
:102E4000DA0108958B3F21F40E94C216819504C0D7
:102E50008C3F29F40E94C2168093DB010895843FC1
:102E600021F48091D701816017C0853F21F48091C2
:102E7000D701826011C0863F21F48091D701846020
:102E80000BC0873F21F48091D701886005C0883F3F
:102E900031F48091D70180618093D70108958D3FEF
:102EA00021F48091D50181600BC08E3F21F4809187
:102EB000D501826005C08F3F29F48091D5018460DF
:102EC0008093D5010895803F39F48091D90187FF1F
:102ED0006CC01092D90169C0813F29F48091D90159
:102EE0001816BCF362C09091D801823F29F497FF75
:102EF0005CC01092D80159C0833F19F41916CCF365
:102F000054C0893F41F48091DA0118160CF04DC08D
:102F10001092DA014AC08A3F29F48091DA0187FFD2
:102F200044C0F6CF8B3F39F48091DB0187FF3DC071
:102F30001092DB013AC08C3F29F48091DB01181616
:102F4000BCF333C0843F21F48091D7018E7F17C03A
:102F5000853F21F48091D7018D7F11C0863F21F4F8
:102F60008091D7018B7F0BC0873F21F48091D701DF
:102F7000877F05C0883F31F48091D7018F7E809391
:102F8000D70113C08D3F21F48091D5018E7F0BC0F6
:102F90008E3F21F48091D5018D7F05C08F3F29F4AC
:102FA0008091D5018B7F8093D5018091D8018111CB
:102FB0000EC08091D90181110AC08091DA0181117E
:102FC00006C08091DB01811102C01092D6010895E4
:102FD00087ED91E00E94FB090E94DE159093D401D9
:102FE0008093D30108951F93CF93DF938091D301F2
:102FF0009091D4010E94EA15AC019091D6019923D9
:1030000021F02091090130E006C020910A018AE0F8
:10301000289F900111244217530708F486C080911D
:10302000D801C091D901D091DA011091DB01811151
:1030300007C0C11176C0D11174C0111172C075C022
:103040009F3F19F09F5F9093D601181624F40E94B9
:1030500079168093D8018091D80187FF05C00E941E
:10306000791681958093D8011C1624F40E94791654
:103070008093D9018091D90187FF05C00E947916FC
:1030800081958093D9016091D801662339F1C0916F
:10309000D901CC2319F1772767FD7095872F972FDA
:1030A0000E94722223E333E343E35FE30E94D622CC
:1030B0000E943A226093D8016C2F772767FD7095A4
:1030C000872F972F0E94722223E333E343E35FE3CA
:1030D0000E94D6220E943A226093D9011D1624F440
:1030E0000E94C2168093DA018091DA0187FF05C041
:1030F0000E94C21681958093DA01111624F40E9471
:10310000C2168093DB018091DB0187FF05C00E941E
:10311000C21681958093DB01DF91CF911F910C94B2
:10312000E8179F3F09F08ECF96CFDF91CF911F9187
:103130000895E7EDF1E085E0DF011D928A95E9F75A
:103140001092D6011092D5010895833081F128F4B0
:10315000813059F08230D1F00895853009F449C0AA
:10316000B8F1863009F456C0089580910A01262FDF
:1031700030E0280F311D2F3F310524F4680F609394
:103180000A0108958FEF80930A0108958091090143
:10319000262F30E0280F311D2F3F310524F4680F12
:1031A0006093090108958FEF80930901089580913C
:1031B0000801262F30E0280F311D2F3F310524F460
:1031C000680F6093080108958FEF809308010895B8
:1031D00080910701262F30E0280F311D2F3F310548
:1031E00024F4680F6093070108958FEF809307011F
:1031F000089580910601262F30E0280F311D2F3FC2
:10320000310524F4680F6093060108958FEF8093D1
:103210000601089580910501262F30E0280F311D09
:103220002F3F310524F4680F6093050108958FEF57
:10323000809305010895833011F128F4813049F01D
:10324000823091F00895853081F120F18630C1F10E
:10325000089580910A01681720F4861B80930A0163
:10326000089510920A01089580910901681720F4C9
:10327000861B809309010895109209010895809199
:103280000801681720F4861B8093080108951092A6
:103290000801089580910701681720F4861B809328
:1032A000070108951092070108958091060168179B
:1032B00020F4861B8093060108951092060108955C
:1032C00080910501681720F4861B809305010895FD
:1032D0001092050108950F931F938D3109F471C069
:1032E00008F045C0803109F485C008F5873009F43D
:1032F0006FC068F4863009F0ADC08091CD01817F48
:103300008E7F8093CD0181E08093DD01A4C08B305E
:1033100009F49EC08E3009F09DC08091CD0182FBE2
:10332000222720F991E0922790FB82F96CC0863128
:1033300009F48EC060F4813109F08CC00E94940EB3
:103340009091020181E089278093020181C0893137
:1033500009F47EC08B3109F07DC08091CD0181FBE5
:10336000222720F991E0922790FB81F94CC0853308
:1033700009F466C048F4873209F462C008F44FC00B
:10338000893209F45DC066C0833438F48A3308F0AA
:1033900044C0883309F45CC05DC0833409F450C074
:1033A000883409F057C00E94940E0FEF13ED20E30C
:1033B000015010402040E1F700C000000E94391683
:1033C00047C00E94F51A0E94E4090E94460640C0C8
:1033D0009091CD01892F8095817080FB90F929F023
:1033E000966098609093CD0136C0997F977F9093B7
:1033F000CD012EC08091CD0183FB222720F991E0E1
:10340000922790FB83F98093CD01992309F1809154
:10341000CD0181608093CD011BC0895301C08D51C6
:1034200041E050E060E070E08A019B0104C0000FC1
:10343000111F221F331F8A95D2F7C901B80104C09A
:1034400061E070E080E090E00E9454120E94940ECF
:1034500081E001C080E01F910F91089580E0089500
:1034600080E008958E518A3030F4E82FF0E0EA5E73
:10347000FE4F8081089580E00895CF93C82F8091FA
:10348000DD01813079F018F08230E9F186C0E091F9
:103490000301F09104018081813169F0823209F0E9
:1034A0007EC009C0E0910301F09104018081813167
:1034B00011F0823261F48C2F0E942E1A811104C007
:1034C0008C2F0E946B191DC081E090E01AC08C2FD8
:1034D0000E94301A811114C0C43179F048F4CB3005
:1034E00079F0C03109F05FC082E08093DD0108C04F
:1034F000C93219F0C83321F056C01092DD0153C013
:1035000081E0817052C0C93281F110F5C43169F196
:10351000A8F4C73009F045C08AE080930A0194E11D
:103520009093090193E0909308018093070188E04C
:103530008093060188E28093050133C082EE8C0FF0
:10354000863078F58C2F0E94321A8093DC0129C0D6
:10355000CE34E9F020F4CB3421F56AE013C0C13554
:1035600079F0C235F1F461E00DC08091DC0188236F
:1035700019F01092DC0115C081E08093DD0115C0C7
:1035800061E006C08091DC010E94A5180AC06AE0D3
:103590008091DC010E941B1904C01092DD0180E0C3
:1035A00004C081E002C080E0ACCFCF910895E1E893
:1035B000F0E08081886080838081816080838FB724
:1035C000F89493E09093890090ED909388008FBFDA
:1035D0000895EFE6F0E08081826080830895EFE651
:1035E000F0E080818D7F80830895EFE6F0E09081A8
:1035F00082E08927808308951F920F920FB60F9261
:1036000011242F933F934F935F936F937F938F93E7
:103610009F93AF93BF93EF93FF938091DE019091BF
:10362000DF0101969093DF018093DE01811103C0D9
:1036300082E00E944606E091DF01E695E695F0E023
:10364000E954FC4FE4918091DE018E1303C080E0C9
:103650000E944606FF91EF91BF91AF919F918F918C
:103660007F916F915F914F913F912F910F900FBE7E
:103670000F901F9018958091F0010895CF93DF93DC
:1036800000D01F92CDB7DEB79C018091F801843045
:1036900019F593E099833B832A839093E9008FEF98
:1036A0009091E800815095FD06C095ED9A95F1F74F
:1036B00000008111F5CF8091E80085FF0DC040E04A
:1036C00050E063E070E0CE0101960E94A71D80915A
:1036D000E8008E778093E8000F900F900F90DF91B5
:1036E000CF910895CF93DF9300D01F92CDB7DEB76F
:1036F0002091F801243021F522E029839B838A83DD
:1037000083E08093E9008FEF9091E800815095FD70
:1037100006C095ED9A95F1F700008111F5CF8091E3
:10372000E80085FF0DC040E050E063E070E0CE01AE
:1037300001960E94A71D8091E8008E778093E80093
:103740000F900F900F90DF91CF9108952091F80185
:103750002430F1F422E02093E9002FEF3091E800CB
:10376000215035FD06C035ED3A95F1F700002111E5
:10377000F5CF2091E80025FF0BC040E050E065E068
:1037800070E00E94A71D8091E8008E778093E8008A
:103790000895CF93DF93EC019091F801943009F0F4
:1037A00046C0809115018823D9F0809102018823B9
:1037B000B9F09093E9008FEF9091E800815095FD6A
:1037C00006C095E19A95F1F700008111F5CF80913F
:1037D000E80085FF2CC040E050E060E170E017C0D9
:1037E00081E08093E9008FEF9091E800815095FD92
:1037F00006C095ED9A95F1F700008111F5CF809103
:10380000E80085FF14C040E050E068E070E0CE01C1
:103810000E94A71D8091E8008E778093E80080E1E8
:10382000FE01A0EEB1E001900D928A95E1F7DF91E3
:10383000CF9108958091F701811109C00E943C1F2A
:103840000E94991F8091E20084608093E2000895B5
:103850001092F701089508950C94E91A0E94CF156B
:103860000E94EF1A0E94E4090C94460642E061ECC3
:1038700081E00E94B61E42E061EC82E00E94B61E2A
:1038800042E061EC83E00E94B61E42E161EC84E01C
:103890000C94B61E8091FA01833009F455C030F4BF
:1038A000813071F0823009F48EC008958A3009F4B5
:1038B0007AC08B3009F460C0893009F09CC020C008
:1038C0008091F901813A09F096C08091E800877FE4
:1038D0008093E8008091FD019091FE01892B21F4F5
:1038E00060E180EE91E003C060E080E090E070E095
:1038F0000E94F21D8091E8008B778093E800089584
:103900008091F901813209F076C08091FD0190919A
:10391000FE01009719F0039709F06DC08091E8004F
:10392000877F8093E8008091E80082FD05C0809148
:10393000F8018111F8CF5FC08091F1008093F00110
:103940008091E8008B7753C08091F901813A09F0AA
:1039500052C08091FD019091FE01892B09F04BC06E
:103960008091E800877F8093E8008091E80080FFE5
:10397000FCCF8091150136C08091F9018132D9F5D3
:103980008091FD019091FE01892BA9F58091E800BD
:10399000877F8093E8000E94EB1E8091FB0180935B
:1039A00015010C94940E8091F901813221F58091DA
:1039B000E800877F8093E8000E94EB1E8091FC0165
:1039C0008093F10108958091F901813AA1F48091E9
:1039D000E800877F8093E8008091E80080FFFCCFBB
:1039E0008091F1018093F1008091E8008E778093BF
:1039F000E8000C94EB1E089584B7877F84BF0FB650
:103A0000F894A8958091600088618093600010927E
:103A100060000FBE80E880936100109261000E94F8
:103A2000330A0E943C1F0E94991F8091E20084602B
:103A30008093E20078940E941F220E94350A8BE056
:103A400091E00E94DF090E94D71A8091F801853029
:103A500069F40E948E158091F6018823B1F30E94CB
:103A6000BB15882391F30E94911DEFCF0E943B0A62
:103A7000ECCF292F332723303105C9F064F42130EE
:103A8000310581F02230310509F043C08DE690E028
:103A90002BE234E042C021323105F1F0223231050F
:103AA00041F137C082E190E028E934E036C099273F
:103AB0008130910541F08230910541F0892B49F523
:103AC000E7E2F4E005C0EFE0F4E002C0E7EFF3E086
:103AD000849190E09F0121C06430D8F4E62FF0E09B
:103AE000EE0FFF1FE45DFE4F2081318189E090E001
:103AF00014C0643070F470E0FB01EE0FFF1FEC5D4A
:103B0000FE4F20813181FB01E05EFE4F808190E01D
:103B100004C080E090E020E030E0FA0131832083AF
:103B2000089580E189BD82E189BD09B400FEFDCF21
:103B30008091D8008F7D8093D8008091E0008260D2
:103B40008093E0008091E00081FDFCCF0895CF924A
:103B5000DF92EF92FF920F931F93CF93DF93EC01CD
:103B60008B016A010E940A1F811133C0C114D10464
:103B700039F0F60180819181081B190BC80FD91FFC
:103B8000E12CF12C0115110519F18091E80085FD5A
:103B900016C08091E8008E778093E800C114D104AC
:103BA00049F0F60180819181E80EF91EF182E082F0
:103BB00085E00FC00E940A1F882321F30AC0899163
:103BC0008093F10001501109FFEFEF1AFF0ADACFDD
:103BD00080E0DF91CF911F910F91FF90EF90DF90E8
:103BE000CF9008952091FF013091000226173707EA
:103BF00048F06115710539F42091E8002E77209383
:103C0000E80001C0B90140E061157105A9F12091FA
:103C1000F801222309F443C0253009F442C0209161
:103C2000E80023FD40C02091E80022FD32C0209131
:103C3000E80020FFE9CF4091F3002091F20030E04E
:103C4000342BFC01CF016115710559F02830310585
:103C500040F481918093F100615071092F5F3F4FD3
:103C6000F1CF41E02830310509F040E02091E80033
:103C70002E772093E800C8CF4111C9CF0AC08091A8
:103C8000F801882361F0853061F08091E80083FDC0
:103C90000AC08091E80082FFF2CF80E0089582E0C0
:103CA000089583E0089581E008952091FF01309107
:103CB00000022617370748F06115710539F4209185
:103CC000E8002E772093E80001C0B901FC0120E054
:103CD0006115710591F18091F801882309F440C0C4
:103CE000853009F43FC08091E80083FD3DC080919C
:103CF000E80082FD2FC08091E80080FFE9CF20918D
:103D0000F3008091F20090E0922B6115710559F05B
:103D10008830910540F424912093F1003196615050
:103D200071090196F2CF21E0089709F020E0809117
:103D3000E8008E778093E800CBCF2111CCCF0AC06A
:103D40008091F801882361F0853061F08091E8006E
:103D500083FD0AC08091E80082FFF2CF80E00895E1
:103D600082E0089583E0089581E00895982F9730C8
:103D700058F59093E900981739F07091EC00209174
:103D8000ED005091F00003C0242F762F50E021FF6A
:103D900019C03091EB003E7F3093EB003091ED0085
:103DA0003D7F3093ED003091EB0031603093EB00BC
:103DB0007093EC002093ED005093F0002091EE0002
:103DC00027FF07C09F5FD3CF8F708093E90081E00A
:103DD000089580E008958091F90187FF11C08091D6
:103DE000E80082FD05C08091F8018111F8CF11C073
:103DF0008091E8008B770BC08091F801882349F00F
:103E00008091E80080FFF8CF8091E8008E77809362
:103E1000E80008952091E4003091E50095E6409196
:103E2000EC00842F817040FF22C08091E80080FD6B
:103E30001CC08091F801882391F0853091F0809129
:103E4000EB0085FD10C04091E4005091E500421761
:103E5000530729F39A01915011F784E0089582E005
:103E6000089583E0089581E0089580E008954091E9
:103E7000E80042FFDECF08950E94AA1F0E94B21FF1
:103E8000E0EEF0E0808181608083E8EDF0E0808109
:103E90008F77808319BCA7EDB0E08C918E7F8C93D7
:103EA00080818F7E80831092F70108950F931F9376
:103EB000CF93DF930E94AA1F0E94B21FC8EDD0E0EB
:103EC00088818F77888388818068888388818F7DC7
:103ED000888319BC1092F8011092F4011092F60137
:103EE0001092F50100EE10E0F80180818B7F808355
:103EF00088818160888342E060E080E00E94B61E95
:103F0000E1EEF0E080818E7F8083E2EEF0E0808160
:103F100081608083808188608083F80180818E7FCA
:103F20008083888180618883DF91CF911F910F9179
:103F30000895E8EDF0E080818F7E8083E7EDF0E08A
:103F400080818160808384E082BF81E08093F7017B
:103F50000C94561FE8EDF0E080818E7F80831092F4
:103F6000E20008951092DA001092E10008951F9285
:103F70000F920FB60F9211242F933F934F935F939D
:103F80006F937F938F939F93AF93BF93EF93FF9321
:103F90008091E10082FF0BC08091E20082FF07C0A8
:103FA0008091E1008B7F8093E1000E941E2280912E
:103FB000DA0080FF1FC08091D80080FF1BC0809175
:103FC000DA008E7F8093DA008091D90080FF0DC0E7
:103FD00080E189BD82E189BD09B400FEFDCF81E0A9
:103FE0008093F8010E941A1C05C019BC1092F801B8
:103FF0000E94281C8091E10080FF19C08091E2009E
:1040000080FF15C08091E2008E7F8093E200809156
:10401000E20080618093E2008091D800806280930A
:10402000D80019BC85E08093F8010E942C1C809177
:10403000E10084FF30C08091E20084FF2CC080E169
:1040400089BD82E189BD09B400FEFDCF8091D80011
:104050008F7D8093D8008091E1008F7E8093E10076
:104060008091E2008F7E8093E2008091E200816087
:104070008093E2008091F401882311F084E007C06E
:104080008091E30087FD02C081E001C083E080935E
:10409000F8010E942E1C8091E10083FF29C08091CD
:1040A000E20083FF25C08091E100877F8093E100DB
:1040B00082E08093F8011092F4018091E1008E7FFC
:1040C0008093E1008091E2008E7F8093E2008091F6
:1040D000E20080618093E20042E060E080E00E94C4
:1040E000B61E8091F00088608093F0000E942B1C27
:1040F000FF91EF91BF91AF919F918F917F916F91C0
:104100005F914F913F912F910F900FBE0F901F9095
:1041100018951F920F920FB60F9211242F933F9371
:104120004F935F936F937F938F939F93AF93BF93BF
:10413000CF93DF93EF93FF93C091E900CF7080910D
:10414000EC00D82FD17080FDD0E81092E90080916A
:10415000F000877F8093F00078940E94CD20109229
:10416000E9008091F00088608093F000CD2BCF7043
:10417000C093E900FF91EF91DF91CF91BF91AF9193
:104180009F918F917F916F915F914F913F912F916F
:104190000F900FBE0F901F9018951F93CF93DF9332
:1041A000CDB7DEB7AA970FB6F894DEBF0FBECDBF6E
:1041B000E9EFF1E088E08E0F9091F10091938E137A
:1041C000FBCF0E944A1C8091E80083FF1FC18091B1
:1041D000F9019091FA01492F50E04A30510508F059
:1041E00015C1FA01E558FF4F0C947F23803881F008
:1041F000823809F00BC18091FD018F708093E90036
:104200008091EB0085FB882780F91092E90006C0B9
:104210008091F5019091F601911182609091E800F2
:10422000977F9093E8008093F1001092F100C8C04E
:10423000282F2D7F09F0EAC0882319F0823061F021
:10424000E5C08091FB01813009F0E0C0933009F0B6
:1042500080E08093F6012BC08091FB01811127C083
:104260008091FD018F7009F4D1C08093E900209105
:10427000EB0020FF1CC0933021F48091EB008062A2
:1042800014C09091EB0090619093EB0021E030E03E
:10429000A90102C0440F551F8A95E2F74093EA0036
:1042A0001092EA008091EB0088608093EB001092FE
:1042B000E9008091E800877F86C08111A7C0109136
:1042C000FB011F778091E3008078812B8093E300CE
:1042D0008091E800877F8093E8000E94EB1E809128
:1042E000E80080FFFCCF8091E30080688093E300CA
:1042F000111102C082E001C083E08093F80186C002
:104300008058823008F082C08091FB019091FC01BE
:104310008C3D53E0950779F583E08A838AE28983AF
:104320004FB7F894DE01139620E03EE051E2E32F10
:10433000F0E050935700E49120FF03C0E295EF7046
:104340003F5FEF708E2F90E0EA3010F0C79601C00B
:10435000C0968D939D932F5F243149F74FBF809175
:10436000E800877F8093E8006AE270E0CE01019662
:104370000E94F21D14C0AE014F5F5F4F6091FD01BE
:104380000E94391DBC01892B09F440C09091E800BE
:10439000977F9093E80089819A810E94551E8091B1
:1043A000E8008B778093E80031C0803879F5809100
:1043B000E800877F8093E8008091F4018093F1000A
:1043C0008091E8008E778093E8000E94EB1E1EC06B
:1043D00081111CC09091FB019230C0F48091E800E3
:1043E000877F8093E8009093F4010E94EB1E8091F8
:1043F000F401811106C08091E30087FD02C081E0D5
:1044000001C084E08093F8010E94361C8091E8008E
:1044100083FF0AC08091E800877F8093E800809145
:10442000EB0080628093EB00AA960FB6F894DEBF93
:104430000FBECDBFDF91CF911F9108950895CF9307
:104440008091F8018823A1F0C091E900CF7090918C
:10445000EC00892F817090FD80E8C82B1092E90054
:104460008091E80083FD0E94CD20CF70C093E900C9
:10447000CF9108950E9441226894B1110C94D022EA
:1044800008950E94B52288F09F5798F0B92F992778
:10449000B751B0F0E1F0660F771F881F991F1AF02F
:1044A000BA95C9F714C0B13091F00E94CF22B1E0A3
:1044B00008950C94CF22672F782F8827B85F39F0A2
:1044C000B93FCCF3869577956795B395D9F73EF4C8
:1044D00090958095709561957F4F8F4F9F4F089570
:1044E000E89409C097FB3EF490958095709561958E
:1044F0007F4F8F4F9F4F9923A9F0F92F96E9BB2744
:104500009395F695879577956795B795F111F8CFBF
:10451000FAF4BB0F11F460FF1BC06F5F7F4F8F4F2A
:104520009F4F16C0882311F096E911C0772321F020
:104530009EE8872F762F05C0662371F096E8862FB8
:1045400070E060E02AF09A95660F771F881FDAF70F
:10455000880F9695879597F9089557FD9058440FC1
:10456000551F59F05F3F71F04795880F97FB991FD2
:1045700061F09F3F79F0879508951216130614068F
:10458000551FF2CF4695F1DF08C01616170618061C
:10459000991FF1CF86957105610508940895E894F7
:1045A000BB2766277727CB0197F908950E94E92258
:1045B0000C945A230E944C2338F00E94532320F07D
:1045C000952311F00C9443230C94492311240C944B
:1045D000D0220E94AD2270F3959FC1F3950F50E059
:1045E000551F629FF001729FBB27F00DB11D639FA5
:1045F000AA27F00DB11DAA1F649F6627B00DA11D4B
:10460000661F829F2227B00DA11D621F739FB00DF0
:10461000A11D621F839FA00D611D221F749F332760
:10462000A00D611D231F849F600D211D822F762FF9
:104630006A2F11249F5750409AF0F1F088234AF0D6
:10464000EE0FFF1FBB1F661F771F881F9150504042
:10465000A9F79E3F510580F00C9443230C94D0227F
:104660005F3FE4F3983ED4F3869577956795B795C9
:10467000F795E7959F5FC1F7FE2B880F911D9695E3
:10468000879597F9089597F99F6780E870E060E053
:1046900008959FEF80EC089500240A9416161706DB
:1046A00018060906089500240A9412161306140623
:1046B00005060895092E0394000C11F4882352F086
:1046C000BB0F40F4BF2B11F460FF04C06F5F7F4F3E
:1046D0008F4F9F4F089597FB072E16F4009407D035
:1046E00077FD09D00E94852307FC05D03EF4909504
:1046F00081959F4F0895709561957F4F0895EE0FB6
:10470000FF1F0590F491E02D0994AA1BBB1B51E1FA
:1047100007C0AA1FBB1FA617B70710F0A61BB70B31
:10472000881F991F5A95A9F780959095BC01CD01D6
:104730000895F999FECF92BD81BDF89A992780B569
:104740000895A8E1B0E042E050E00C94C023262F89
:10475000F999FECF92BD81BDF89A019700B4021677
:1047600031F020BD0FB6F894FA9AF99A0FBE089569
:104770000196272F0E94A8230C94A723DC01CB01CC
:10478000FC01F999FECF06C0F2BDE1BDF89A319661
:1047900000B40D9241505040B8F70895F894FFCFFF
:1047A000052001BA0128080A03140A3B1BC91BA6ED
:1047B0001B721B3E1B0101020304050607080900CA
:1047C000404D363966051905E304AA043D04560434
:0447D0006F048804E6
:00000001FF
